:020000003128A5
:1000080009008A0182002F345934313452340034C3
:100018008A012808A80A82002F3413340034553482
:10002800163400343134193400344334213456340E
:100038006E280D3463280034003455347C28443449
:1000480083285A3471283034722831347428323471
:10005800762833347828003400348316203085001D
:10006800083081000030900000309F008312163065
:100078009800073099000516FA308F210512A0164E
:100088004930CF00A001A1018512D70189200000C5
:100098001A211030A8002F21AB000C20003A0319B8
:1000A8005D282B0603195A28A80A51280C20A800F5
:1000B8004F280C20003A031D4B283F303C21672075
:1000C8006920C6204B280D303C2905160A308F219F
:1000D80005120800663003216328000000307928E3
:1000E80001307928023079280330D7008920632825
:1000F800D70A5708043A0319D70189206328D70378
:100108000330D71BD700892063285708A30005119F
:100118008510A303A31B080005118514A303A31BC3
:10012800080005158514A303A31B080005158510F1
:100138000800D4000530D3005408A820201A08006D
:100148006720D30BA0280800AB20D1200800D600D8
:10015800C220B301851EAC289821B30BAE28851E9A
:10016800AC288316851283125608D60A0520A300E8
:10017800003A0319080023083C21B828C6203F3953
:10018800013E9F294F08D0075008D1070310D10C12
:100198000318D1175108CF070800C901201264308D
:1001A800D5009A215A21A3002018DD28D50BD5287F
:1001B800080049080A3A0319D1284908353E84003D
:1001C80023088000C90A0D3A031DD328C901201647
:1001D8000800AE012F21A3003030A302031C01291F
:1001E8000A302302031801290310AE0D2E08AE0DA4
:1001F800AE0DAE072308AE07EE282E080800A011A2
:10020800A40064300B210A300B21A0150130A50091
:100218003030A9002508A402031C1529A90AA01535
:100228000F29A4072908A0193C210800C9015A214F
:10023800201C1B296400A3004908123A03194B2803
:1002480035304907C90A8400230880000D3A031D88
:100258001B29C901080035304907C90A840000086C
:100268000800FF30B107031CB20732083104080048
:10027800AE00851201308F2104304E2102304E210C
:100288000830B1000130AE0D031803304E21B10B18
:1002980046290800A3009A218316851283129A2101
:1002A800A30B53298316851683120800A01020106B
:1002B800851A080072217221A2000830B100AE012F
:1002C800722103197029A3002208A302AE0DB10BF5
:1002D80064292E0820140800A0140800A301A30A0A
:1002E80003190800000000000000000000000000E2
:1002F80000000000851A7329A301A30A0319080046
:1003080000000000000000000000000000002308BA
:10031800851E81290800B0009E21B00B9029080095
:1003280001309F2902309F2905309F290A309F29D3
:1003380032309F296430AF00000000000000000048
:0C034800000000000000AF0BA02908001E
:02400E00E4309C
:00000001FF
